
ADC motor.elf:     file format elf32-avr

Sections:
Idx Name          Size      VMA       LMA       File off  Algn
  0 .text         0000006c  00000000  00000000  00000054  2**1
                  CONTENTS, ALLOC, LOAD, READONLY, CODE
  1 .data         00000000  00800060  00800060  000002b8  2**0
                  ALLOC, LOAD, DATA
  2 .comment      0000002f  00000000  00000000  000002b8  2**0
                  CONTENTS, READONLY
  3 .debug_aranges 00000038  00000000  00000000  000002e7  2**0
                  CONTENTS, READONLY, DEBUGGING
  4 .debug_info   00000b0e  00000000  00000000  0000031f  2**0
                  CONTENTS, READONLY, DEBUGGING
  5 .debug_abbrev 00000600  00000000  00000000  00000e2d  2**0
                  CONTENTS, READONLY, DEBUGGING
  6 .debug_line   000003c7  00000000  00000000  0000142d  2**0
                  CONTENTS, READONLY, DEBUGGING
  7 .debug_frame  00000060  00000000  00000000  000017f4  2**2
                  CONTENTS, READONLY, DEBUGGING
  8 .debug_str    00000196  00000000  00000000  00001854  2**0
                  CONTENTS, READONLY, DEBUGGING
  9 .debug_loc    00000377  00000000  00000000  000019ea  2**0
                  CONTENTS, READONLY, DEBUGGING
 10 .debug_ranges 00000028  00000000  00000000  00001d61  2**0
                  CONTENTS, READONLY, DEBUGGING
 11 .text         00000004  00000260  00000260  000002b4  2**1
                  CONTENTS, ALLOC, LOAD, READONLY, CODE
 12 .note.gnu.avr.deviceinfo 0000003c  00000000  00000000  00001d8c  2**2
                  CONTENTS, READONLY, DEBUGGING
 13 .text.command 00000016  0000024a  0000024a  0000029e  2**1
                  CONTENTS, ALLOC, LOAD, READONLY, CODE
 14 .text.data    00000018  00000232  00000232  00000286  2**1
                  CONTENTS, ALLOC, LOAD, READONLY, CODE
 15 .text.main    00000176  0000006c  0000006c  000000c0  2**1
                  CONTENTS, ALLOC, LOAD, READONLY, CODE
 16 .text.libgcc.div 00000028  000001e2  000001e2  00000236  2**1
                  CONTENTS, ALLOC, LOAD, READONLY, CODE
 17 .text.libgcc.div 00000028  0000020a  0000020a  0000025e  2**1
                  CONTENTS, ALLOC, LOAD, READONLY, CODE

Disassembly of section .text:

00000000 <__vectors>:
   0:	0c 94 2a 00 	jmp	0x54	; 0x54 <__ctors_end>
   4:	0c 94 30 01 	jmp	0x260	; 0x260 <__bad_interrupt>
   8:	0c 94 30 01 	jmp	0x260	; 0x260 <__bad_interrupt>
   c:	0c 94 30 01 	jmp	0x260	; 0x260 <__bad_interrupt>
  10:	0c 94 30 01 	jmp	0x260	; 0x260 <__bad_interrupt>
  14:	0c 94 30 01 	jmp	0x260	; 0x260 <__bad_interrupt>
  18:	0c 94 30 01 	jmp	0x260	; 0x260 <__bad_interrupt>
  1c:	0c 94 30 01 	jmp	0x260	; 0x260 <__bad_interrupt>
  20:	0c 94 30 01 	jmp	0x260	; 0x260 <__bad_interrupt>
  24:	0c 94 30 01 	jmp	0x260	; 0x260 <__bad_interrupt>
  28:	0c 94 30 01 	jmp	0x260	; 0x260 <__bad_interrupt>
  2c:	0c 94 30 01 	jmp	0x260	; 0x260 <__bad_interrupt>
  30:	0c 94 30 01 	jmp	0x260	; 0x260 <__bad_interrupt>
  34:	0c 94 30 01 	jmp	0x260	; 0x260 <__bad_interrupt>
  38:	0c 94 30 01 	jmp	0x260	; 0x260 <__bad_interrupt>
  3c:	0c 94 30 01 	jmp	0x260	; 0x260 <__bad_interrupt>
  40:	0c 94 30 01 	jmp	0x260	; 0x260 <__bad_interrupt>
  44:	0c 94 30 01 	jmp	0x260	; 0x260 <__bad_interrupt>
  48:	0c 94 30 01 	jmp	0x260	; 0x260 <__bad_interrupt>
  4c:	0c 94 30 01 	jmp	0x260	; 0x260 <__bad_interrupt>
  50:	0c 94 30 01 	jmp	0x260	; 0x260 <__bad_interrupt>

00000054 <__ctors_end>:
  54:	11 24       	eor	r1, r1
  56:	1f be       	out	0x3f, r1	; 63
  58:	cf e5       	ldi	r28, 0x5F	; 95
  5a:	d8 e0       	ldi	r29, 0x08	; 8
  5c:	de bf       	out	0x3e, r29	; 62
  5e:	cd bf       	out	0x3d, r28	; 61
  60:	0e 94 36 00 	call	0x6c	; 0x6c <_etext>
  64:	0c 94 34 00 	jmp	0x68	; 0x68 <_exit>

00000068 <_exit>:
  68:	f8 94       	cli

0000006a <__stop_program>:
  6a:	ff cf       	rjmp	.-2      	; 0x6a <__stop_program>

Disassembly of section .text:

00000260 <__bad_interrupt>:
 260:	0c 94 00 00 	jmp	0	; 0x0 <__vectors>

Disassembly of section .text.command:

0000024a <command>:
	}
	}
}

void command(unsigned char a){
	PORTD=a;
 24a:	82 bb       	out	0x12, r24	; 18
	PORTC=0x02; //RS=0 and EN=1
 24c:	82 e0       	ldi	r24, 0x02	; 2
 24e:	85 bb       	out	0x15, r24	; 21
	#else
		//round up by default
		__ticks_dc = (uint32_t)(ceil(fabs(__tmp)));
	#endif

	__builtin_avr_delay_cycles(__ticks_dc);
 250:	8f e1       	ldi	r24, 0x1F	; 31
 252:	9e e4       	ldi	r25, 0x4E	; 78
 254:	01 97       	sbiw	r24, 0x01	; 1
 256:	f1 f7       	brne	.-4      	; 0x254 <command+0xa>
 258:	00 c0       	rjmp	.+0      	; 0x25a <command+0x10>
 25a:	00 00       	nop
	_delay_ms(10);
	PORTC=0x00;//RS=0 and EN=0
 25c:	15 ba       	out	0x15, r1	; 21
 25e:	08 95       	ret

Disassembly of section .text.data:

00000232 <data>:
}

void data(unsigned char b){
	PORTD=b;
 232:	82 bb       	out	0x12, r24	; 18
	PORTC=0x03; //RS=1
 234:	83 e0       	ldi	r24, 0x03	; 3
 236:	85 bb       	out	0x15, r24	; 21
 238:	8f e1       	ldi	r24, 0x1F	; 31
 23a:	9e e4       	ldi	r25, 0x4E	; 78
 23c:	01 97       	sbiw	r24, 0x01	; 1
 23e:	f1 f7       	brne	.-4      	; 0x23c <data+0xa>
 240:	00 c0       	rjmp	.+0      	; 0x242 <data+0x10>
 242:	00 00       	nop
	_delay_ms(10);
	PORTC=0x01; //EN=0 and RS=1
 244:	81 e0       	ldi	r24, 0x01	; 1
 246:	85 bb       	out	0x15, r24	; 21
 248:	08 95       	ret

Disassembly of section .text.main:

0000006c <main>:
void data(unsigned char);
void display(char *p);

int main(void){
	int a,b,x=1234,y=0,z,p,q,r,s,sw1;
	DDRA=0x00;
  6c:	1a ba       	out	0x1a, r1	; 26
	DDRD=0xFF;
  6e:	8f ef       	ldi	r24, 0xFF	; 255
  70:	81 bb       	out	0x11, r24	; 17
	DDRC=0x03;
  72:	93 e0       	ldi	r25, 0x03	; 3
  74:	94 bb       	out	0x14, r25	; 20
	DDRB=0xFF;
  76:	87 bb       	out	0x17, r24	; 23
	ADCSRA=0xD7;
  78:	87 ed       	ldi	r24, 0xD7	; 215
  7a:	86 b9       	out	0x06, r24	; 6
	
	command(0x38);
  7c:	88 e3       	ldi	r24, 0x38	; 56
  7e:	0e 94 25 01 	call	0x24a	; 0x24a <command>
	command(0x80);
  82:	80 e8       	ldi	r24, 0x80	; 128
  84:	0e 94 25 01 	call	0x24a	; 0x24a <command>
	command(0x0f);
  88:	8f e0       	ldi	r24, 0x0F	; 15
  8a:	0e 94 25 01 	call	0x24a	; 0x24a <command>
	command(0x06);
  8e:	86 e0       	ldi	r24, 0x06	; 6
  90:	0e 94 25 01 	call	0x24a	; 0x24a <command>
	command(0x01);
  94:	81 e0       	ldi	r24, 0x01	; 1
  96:	0e 94 25 01 	call	0x24a	; 0x24a <command>
	
	while(1){
		command(0x80);
  9a:	80 e8       	ldi	r24, 0x80	; 128
  9c:	0e 94 25 01 	call	0x24a	; 0x24a <command>
		ADCSRA=0xD7;
  a0:	87 ed       	ldi	r24, 0xD7	; 215
  a2:	86 b9       	out	0x06, r24	; 6
		ADCSRA=0x40;
  a4:	80 e4       	ldi	r24, 0x40	; 64
  a6:	86 b9       	out	0x06, r24	; 6
		ADMUX=0x00;
  a8:	17 b8       	out	0x07, r1	; 7
		while(ADCSRA&0x40==0x40);
  aa:	30 99       	sbic	0x06, 0	; 6
  ac:	fe cf       	rjmp	.-4      	; 0xaa <main+0x3e>
		a=ADCL;
  ae:	84 b1       	in	r24, 0x04	; 4
		a|=(ADCH<<8);
  b0:	c5 b1       	in	r28, 0x05	; 5
  b2:	d0 e0       	ldi	r29, 0x00	; 0
  b4:	dc 2f       	mov	r29, r28
  b6:	cc 27       	eor	r28, r28
  b8:	c8 2b       	or	r28, r24
		p=a/1000;
  ba:	ce 01       	movw	r24, r28
  bc:	68 ee       	ldi	r22, 0xE8	; 232
  be:	73 e0       	ldi	r23, 0x03	; 3
  c0:	0e 94 f1 00 	call	0x1e2	; 0x1e2 <__divmodhi4>
  c4:	8c 01       	movw	r16, r24
		data(p+48);
  c6:	80 e3       	ldi	r24, 0x30	; 48
  c8:	86 0f       	add	r24, r22
  ca:	0e 94 19 01 	call	0x232	; 0x232 <data>
  ce:	8f e5       	ldi	r24, 0x5F	; 95
  d0:	9a ee       	ldi	r25, 0xEA	; 234
  d2:	01 97       	sbiw	r24, 0x01	; 1
  d4:	f1 f7       	brne	.-4      	; 0xd2 <main+0x66>
  d6:	00 c0       	rjmp	.+0      	; 0xd8 <main+0x6c>
  d8:	00 00       	nop
		_delay_ms(30);
		q=(a%1000);
		y=q;
		q=q/100;
  da:	c8 01       	movw	r24, r16
  dc:	64 e6       	ldi	r22, 0x64	; 100
  de:	70 e0       	ldi	r23, 0x00	; 0
  e0:	0e 94 f1 00 	call	0x1e2	; 0x1e2 <__divmodhi4>
  e4:	8c 01       	movw	r16, r24
		data(q+48);
  e6:	80 e3       	ldi	r24, 0x30	; 48
  e8:	86 0f       	add	r24, r22
  ea:	0e 94 19 01 	call	0x232	; 0x232 <data>
		y=(y%100);
		s=y;
		y=y/10;
  ee:	c8 01       	movw	r24, r16
  f0:	6a e0       	ldi	r22, 0x0A	; 10
  f2:	70 e0       	ldi	r23, 0x00	; 0
  f4:	0e 94 f1 00 	call	0x1e2	; 0x1e2 <__divmodhi4>
  f8:	18 2f       	mov	r17, r24
		data(y+48);
  fa:	80 e3       	ldi	r24, 0x30	; 48
  fc:	86 0f       	add	r24, r22
  fe:	0e 94 19 01 	call	0x232	; 0x232 <data>
		r=(s%10);
		data(r+48);
 102:	80 e3       	ldi	r24, 0x30	; 48
 104:	81 0f       	add	r24, r17
 106:	0e 94 19 01 	call	0x232	; 0x232 <data>
 10a:	8f e5       	ldi	r24, 0x5F	; 95
 10c:	9a ee       	ldi	r25, 0xEA	; 234
 10e:	01 97       	sbiw	r24, 0x01	; 1
 110:	f1 f7       	brne	.-4      	; 0x10e <main+0xa2>
 112:	00 c0       	rjmp	.+0      	; 0x114 <main+0xa8>
 114:	00 00       	nop
		_delay_ms(30);
		command(0x01);
 116:	81 e0       	ldi	r24, 0x01	; 1
 118:	0e 94 25 01 	call	0x24a	; 0x24a <command>
		if(a>700){
 11c:	cd 3b       	cpi	r28, 0xBD	; 189
 11e:	d2 40       	sbci	r29, 0x02	; 2
 120:	3c f0       	brlt	.+14     	; 0x130 <main+0xc4>
			PORTB|=0x05;
 122:	88 b3       	in	r24, 0x18	; 24
 124:	85 60       	ori	r24, 0x05	; 5
 126:	88 bb       	out	0x18, r24	; 24
			PORTB&=~(0x02);
 128:	88 b3       	in	r24, 0x18	; 24
 12a:	8d 7f       	andi	r24, 0xFD	; 253
 12c:	88 bb       	out	0x18, r24	; 24
 12e:	06 c0       	rjmp	.+12     	; 0x13c <main+0xd0>
		}
		else{
			PORTB|=0x06;
 130:	88 b3       	in	r24, 0x18	; 24
 132:	86 60       	ori	r24, 0x06	; 6
 134:	88 bb       	out	0x18, r24	; 24
			PORTB&=~(0X01);
 136:	88 b3       	in	r24, 0x18	; 24
 138:	8e 7f       	andi	r24, 0xFE	; 254
 13a:	88 bb       	out	0x18, r24	; 24
		}
		
		
	//2nd  Motor
	command(0xC0);
 13c:	80 ec       	ldi	r24, 0xC0	; 192
 13e:	0e 94 25 01 	call	0x24a	; 0x24a <command>
	ADCSRA=0xD7;
 142:	87 ed       	ldi	r24, 0xD7	; 215
 144:	86 b9       	out	0x06, r24	; 6
	ADCSRA=0x40;
 146:	80 e4       	ldi	r24, 0x40	; 64
 148:	86 b9       	out	0x06, r24	; 6
	ADMUX=0x01;
 14a:	81 e0       	ldi	r24, 0x01	; 1
 14c:	87 b9       	out	0x07, r24	; 7
	while(ADCSRA&0x40==0x40);
 14e:	30 99       	sbic	0x06, 0	; 6
 150:	fe cf       	rjmp	.-4      	; 0x14e <main+0xe2>
	a=ADCL;
 152:	84 b1       	in	r24, 0x04	; 4
	a|=(ADCH<<8);
 154:	c5 b1       	in	r28, 0x05	; 5
 156:	d0 e0       	ldi	r29, 0x00	; 0
 158:	dc 2f       	mov	r29, r28
 15a:	cc 27       	eor	r28, r28
 15c:	c8 2b       	or	r28, r24
	p=a/1000;
 15e:	ce 01       	movw	r24, r28
 160:	68 ee       	ldi	r22, 0xE8	; 232
 162:	73 e0       	ldi	r23, 0x03	; 3
 164:	0e 94 f1 00 	call	0x1e2	; 0x1e2 <__divmodhi4>
 168:	8c 01       	movw	r16, r24
	data(p+48);
 16a:	80 e3       	ldi	r24, 0x30	; 48
 16c:	86 0f       	add	r24, r22
 16e:	0e 94 19 01 	call	0x232	; 0x232 <data>
 172:	8f e5       	ldi	r24, 0x5F	; 95
 174:	9a ee       	ldi	r25, 0xEA	; 234
 176:	01 97       	sbiw	r24, 0x01	; 1
 178:	f1 f7       	brne	.-4      	; 0x176 <main+0x10a>
 17a:	00 c0       	rjmp	.+0      	; 0x17c <main+0x110>
 17c:	00 00       	nop
	_delay_ms(30);
	q=(a%1000);
	y=q;
	q=q/100;
 17e:	c8 01       	movw	r24, r16
 180:	64 e6       	ldi	r22, 0x64	; 100
 182:	70 e0       	ldi	r23, 0x00	; 0
 184:	0e 94 f1 00 	call	0x1e2	; 0x1e2 <__divmodhi4>
 188:	8c 01       	movw	r16, r24
	data(q+48);
 18a:	80 e3       	ldi	r24, 0x30	; 48
 18c:	86 0f       	add	r24, r22
 18e:	0e 94 19 01 	call	0x232	; 0x232 <data>
	y=(y%100);
	s=y;
	y=y/10;
 192:	c8 01       	movw	r24, r16
 194:	6a e0       	ldi	r22, 0x0A	; 10
 196:	70 e0       	ldi	r23, 0x00	; 0
 198:	0e 94 f1 00 	call	0x1e2	; 0x1e2 <__divmodhi4>
 19c:	18 2f       	mov	r17, r24
	data(y+48);
 19e:	80 e3       	ldi	r24, 0x30	; 48
 1a0:	86 0f       	add	r24, r22
 1a2:	0e 94 19 01 	call	0x232	; 0x232 <data>
	r=(s%10);
	data(r+48);
 1a6:	80 e3       	ldi	r24, 0x30	; 48
 1a8:	81 0f       	add	r24, r17
 1aa:	0e 94 19 01 	call	0x232	; 0x232 <data>
 1ae:	8f e5       	ldi	r24, 0x5F	; 95
 1b0:	9a ee       	ldi	r25, 0xEA	; 234
 1b2:	01 97       	sbiw	r24, 0x01	; 1
 1b4:	f1 f7       	brne	.-4      	; 0x1b2 <main+0x146>
 1b6:	00 c0       	rjmp	.+0      	; 0x1b8 <main+0x14c>
 1b8:	00 00       	nop
	_delay_ms(30);
	command(0x01);
 1ba:	81 e0       	ldi	r24, 0x01	; 1
 1bc:	0e 94 25 01 	call	0x24a	; 0x24a <command>
	if(a>700){
 1c0:	cd 3b       	cpi	r28, 0xBD	; 189
 1c2:	d2 40       	sbci	r29, 0x02	; 2
 1c4:	3c f0       	brlt	.+14     	; 0x1d4 <main+0x168>
		PORTB|=0x28;
 1c6:	88 b3       	in	r24, 0x18	; 24
 1c8:	88 62       	ori	r24, 0x28	; 40
 1ca:	88 bb       	out	0x18, r24	; 24
		PORTB&=~(0x10);
 1cc:	88 b3       	in	r24, 0x18	; 24
 1ce:	8f 7e       	andi	r24, 0xEF	; 239
 1d0:	88 bb       	out	0x18, r24	; 24
 1d2:	63 cf       	rjmp	.-314    	; 0x9a <main+0x2e>
	}
	else{
		PORTB|=0x18;
 1d4:	88 b3       	in	r24, 0x18	; 24
 1d6:	88 61       	ori	r24, 0x18	; 24
 1d8:	88 bb       	out	0x18, r24	; 24
		PORTB&=~(0x20);
 1da:	88 b3       	in	r24, 0x18	; 24
 1dc:	8f 7d       	andi	r24, 0xDF	; 223
 1de:	88 bb       	out	0x18, r24	; 24
 1e0:	5c cf       	rjmp	.-328    	; 0x9a <main+0x2e>

Disassembly of section .text.libgcc.div:

000001e2 <__divmodhi4>:
 1e2:	97 fb       	bst	r25, 7
 1e4:	07 2e       	mov	r0, r23
 1e6:	16 f4       	brtc	.+4      	; 0x1ec <__divmodhi4+0xa>
 1e8:	00 94       	com	r0
 1ea:	07 d0       	rcall	.+14     	; 0x1fa <__divmodhi4_neg1>
 1ec:	77 fd       	sbrc	r23, 7
 1ee:	09 d0       	rcall	.+18     	; 0x202 <__divmodhi4_neg2>
 1f0:	0e 94 05 01 	call	0x20a	; 0x20a <__udivmodhi4>
 1f4:	07 fc       	sbrc	r0, 7
 1f6:	05 d0       	rcall	.+10     	; 0x202 <__divmodhi4_neg2>
 1f8:	3e f4       	brtc	.+14     	; 0x208 <__divmodhi4_exit>

000001fa <__divmodhi4_neg1>:
 1fa:	90 95       	com	r25
 1fc:	81 95       	neg	r24
 1fe:	9f 4f       	sbci	r25, 0xFF	; 255
 200:	08 95       	ret

00000202 <__divmodhi4_neg2>:
 202:	70 95       	com	r23
 204:	61 95       	neg	r22
 206:	7f 4f       	sbci	r23, 0xFF	; 255

00000208 <__divmodhi4_exit>:
 208:	08 95       	ret

Disassembly of section .text.libgcc.div:

0000020a <__udivmodhi4>:
 20a:	aa 1b       	sub	r26, r26
 20c:	bb 1b       	sub	r27, r27
 20e:	51 e1       	ldi	r21, 0x11	; 17
 210:	07 c0       	rjmp	.+14     	; 0x220 <__udivmodhi4_ep>

00000212 <__udivmodhi4_loop>:
 212:	aa 1f       	adc	r26, r26
 214:	bb 1f       	adc	r27, r27
 216:	a6 17       	cp	r26, r22
 218:	b7 07       	cpc	r27, r23
 21a:	10 f0       	brcs	.+4      	; 0x220 <__udivmodhi4_ep>
 21c:	a6 1b       	sub	r26, r22
 21e:	b7 0b       	sbc	r27, r23

00000220 <__udivmodhi4_ep>:
 220:	88 1f       	adc	r24, r24
 222:	99 1f       	adc	r25, r25
 224:	5a 95       	dec	r21
 226:	a9 f7       	brne	.-22     	; 0x212 <__udivmodhi4_loop>
 228:	80 95       	com	r24
 22a:	90 95       	com	r25
 22c:	bc 01       	movw	r22, r24
 22e:	cd 01       	movw	r24, r26
 230:	08 95       	ret
